:1000000008308A003B2E00000A108A100A1182076D
:100010005334743461347234743420344C346F3457
:10002000673420344D34653474346534723421348B
:1000300000340A108A100A1182074D3461346E347C
:10004000753461346C3420344D346F346434653429
:1000500000340A108A100A118207523465346D3454
:100060006F347434653420344D346F346434653403
:1000700000340A108A100A11820749346E34693438
:100080007434693461346C3469347A3465340034DE
:100090000A108A100A11820743346D346434203404
:1000A0004534723472346F3472343F3400340A1081
:1000B0008A100A11820720342534303435342E3426
:1000C0003334663420346B3448347A3400344C3062
:1000D0008400000803197B280330F800F701F70BB0
:1000E0006F28F80B6E283C30F700F70B75280000DE
:1000F0000000800B6C2800344B08F039CC00060857
:100100000F394C0486008610061006150611533070
:10011000F700F70B89280034F0308316860083122D
:100120000610861406150608F039EA0006110615B1
:100130000608F039EB0006110030831686008312A2
:100140006B0EF7000F30F70577086A04F8000034EB
:100150005308D4005408F039D50006080F39550467
:1001600086008610061006150611D40EF030D40550
:1001700006080F3954048600061506118C207808ED
:10018000D400D41BBE28003400308316860005300E
:100190008312CC0067203030CB007C203030CB0085
:1001A0007C203030CB007C202030CB007C202E30D7
:1001B000D300A8200830D300A8200D30D300A820F9
:1001C0000630D300A8208A150A12762E6908F03965
:1001D000EA0006080F396A04860086100614061520
:1001E0000611E90EF030E90506080F3969048600AA
:1001F000061506118C207808EA00EA1BFA2800345C
:100200000130D300A8208A150A12BB2E8E30F700C9
:100210005808F8005708F900FA01F808031D1A29D0
:100220007908F800F9010830F702F808031D1A29C7
:10023000F70122290310F81B2129F90DF80DF70306
:100240001A29F81300000034530803199529DB001C
:10025000570803199529DB07031C2F2936297F30FE
:10026000DB02031C9529031995293A298130DB0704
:10027000031895295B08F700F801F901FA01540801
:10028000DF00DF175508DE005608DD001830DB0000
:10029000DC015D1C63295A08FA07031C5529F90A79
:1002A000031D5529F80A0319DC175908F907031C1F
:1002B0005C29F80A0319DC175808D500D51755082A
:1002C000F8070318DC17DC0DF80CF90CFA0CDF0C3E
:1002D000DE0CDD0C0310DB0B48290130F707031897
:1002E0009529F81B7A29DF0DFA0DF90DF80DF703A2
:1002F00003199529DF1F8B29FA0A031D8B29F90A97
:10030000031D8B29F80A031D8B29F80CF90CFA0C34
:10031000F70A031995295408DC005808DC06DC1F8D
:100320009329F8179929F8139929F701F801F90188
:10033000FA010000003480308318E006E501E60190
:100340005C08E4006008E4065B080319892AE300FE
:10035000F7005F080319922AE30203192F2A0318F2
:10036000B229EE296008E900E9176108E80062088F
:10037000E700E6010310E90CE80CE70CE60CE30BE0
:10038000B929E41FC6296514A62A651063106516ED
:100390005E308400BC2A6512E41BD829631CE32963
:1003A000E90CE80CE70CE60CF70A0319A12AE3298B
:1003B000E91BE6290310E60DE70DE80DE90DF7034B
:1003C0000319A12AD82965174E2A65135C08E40091
:1003D000DC1FEC29E9179A2AE9139A2A5F08E3003F
:1003E000F7005B08E3025C08E900E9175D08E80034
:1003F0005E08E700E6010310E90CE80CE70CE60CE8
:10040000E30BFA29E41F072AE514A62AE510631076
:10041000E51662308400BC2AE512E41B192A631C2D
:10042000242AE90CE80CE70CE60CF70A0319A12AC8
:10043000242AE91B272A0310E60DE70DE80DE90D34
:10044000F7030319A12A192AE5174E2AE5136008B4
:10045000E400E01F2D2AE9179A2AE9139A2A600876
:10046000E900E9176108E8006208E700E41F3C2A98
:10047000E9136515A62A6511E60163105E30840054
:10048000BC2AE41B642A5C08E400631C4E2AE90CC5
:10049000E80CE70CE60CF70A0319A12AE61F5F2A0D
:1004A000E70A031D5F2AE80A031D5F2AE90A031D04
:1004B0005F2AE90CE80CE70CF70A0319A12A651B6F
:1004C000E529E51B262A832A8030E906E91F6C2AE4
:1004D000A62A6008E400792A5C08E400E908031D04
:1004E000792AE808031D792AE708031D792AF7010C
:1004F0009A2AE91B832A0310E60DE70DE80DE90DA2
:10050000F70B792AA12AE41F872AE9179A2AE91307
:100510009A2A5F08F7006008E9006108E8006208AD
:10052000E7009A2A5B08F7005C08E9005D08E8002C
:100530005E08E7006908F8006808F9006708FA0033
:10054000DB2AF701F801F901FA01DB2AE601E709E4
:10055000E809E909E609E60A031DB52AE70A031DC9
:10056000B52AE80A031DB52AE90A6518C529E51860
:10057000062A65193B2A692A0008E707031CC62AD0
:10058000E80A031DC62AE90A031963148403000854
:10059000E807031CCE2AE90A031963148403000840
:1005A000801BD32A803AE90703186314651ACB2904
:1005B000E51A0C2A412A000000344C08D3005008E8
:1005C000D306D31FE82A03110310CC1B03141B2BE3
:1005D0004C08D3004F08D4004B08D4020319F62A64
:1005E000D31F1B2B0308013A83001B2B5008D40098
:1005F0004C08D4020319022BD31F1B2B0308013A0A
:1006000083001B2B5108D4004D08D40203190E2B74
:10061000D31F1B2B0308013A83001B2B5208D40065
:100620004E08D40203191A2BD31F1B2B0308013ABF
:1006300083001B2B0310003453080319E22BDF0047
:1006400057080319E22BDF020318272B2C2B7F30CE
:10065000DF070318E22B322B8130DF02031CE22B71
:100660000319E22B5F08F700F801F901FA01DE0136
:100670005408DD00DD175508DC005608DB00193092
:10068000DF005A08DB020318552B0130DC02031887
:10069000552BDD020318552BDE020318552BDE0AFD
:1006A000DD0ADC0A5A08DB07872B5908DC0203182D
:1006B000702B0130DD020318702BDE020318702B43
:1006C000DE0ADD0A5908DC075A08DB07031C872B02
:1006D000DC0A031D872BDD0A031D872BDE0A872B0F
:1006E00058088038DD020318862B0130DE0203181B
:1006F000862BDE0A58088038DD075908DC07031C02
:10070000642BDD0A031D642BDE0A642B7A14DF0BD5
:100710008A2B952B0310DB0DDC0DDD0DDE0D031098
:10072000FA0DF90DF80DE00D412B601C9D2B031007
:10073000F80CF90CFA0CE00CA02BF7030319E22BD0
:10074000E01BC92B0310DB0DDC0DDD0DDE0D5A089F
:10075000DB020318B52B0130DC020318B52BDD02D8
:100760000318B52BDE02031CD82B5908DC02031832
:10077000C02B0130DD020318C02BDE02031CD82B76
:1007800058088038DD020318C92B0130DE02031C33
:10079000D82BFA0A031DD82BF90A031DD82BF80A07
:1007A000031DD82BF70A0319E22BF80CF90CFA0CED
:1007B0005408DF005808DF06DF1FE02BF817E62B90
:1007C000F813E62BF701F801F901FA0100000034F3
:1007D0008E30F7004B08F7024C08F9004D08F8007E
:1007E000F917F7080319FF2B0310F908031DFB2B5A
:1007F000F8080319FF2BF90CF80CF70BF42BCC1F9E
:10080000062CF809F909F80A0319F90A000000345E
:100810005B08E4005C08E500E601D81F112C6417B2
:10082000E503D81757080319B42C7F305702031C6F
:10083000702CD700E7010430E8000310DA0DD90D61
:10084000D80DE60DE80B1D2C043057020318302C90
:1008500003305702031DAA2C0A306602031CAA2C7F
:100860000330D702E70A77250310DA0DD90DD80D2A
:10087000E60D60250230E8000310E60CD80CD90C18
:10088000DA0CE80B3C2C77250430E8000310DB0C75
:10089000DC0CDD0CDE0CE80B462C602577255D08B2
:1008A000DE005C08DD005B08DC00DB0160257725ED
:1008B0005C08DE005B08DD00DB01DC016025E61979
:1008C000242CD708031D692CDA0AD90AD80AE60AAB
:1008D000AA2C0310DA0DD90DD80DE60DD703242C60
:1008E000D709D70A7F30D707E7010430E8000310A3
:1008F000DA0DD90DD80DE60DE80B772C0430D707AB
:1009000005305702031CB62C77250310DA0DD90DDC
:10091000D80DE60D0310DA0DD90DD80DE60D6025C2
:100920000310DA0DD90DD80DE60DE70A0330E80003
:100930000310E60CD80CD90CDA0CE80B982C033019
:10094000D702661E802C0310E60CD80CD90CDA0CEA
:10095000D703802CD709D70A0330D707670AE502E7
:10096000031CE5010130B72C0230B72C0030E00049
:10097000E41BC42CE51BC42CE5080319C42C20304F
:10098000E900E620E50BBF2C641FC92C2D30E900DF
:10099000E620E41FD52CE51BD52CE5080319D52C42
:1009A0003030E900E620E50BCD2CE4136413601C25
:1009B000E02C6708E0006708E200640AE207082DFF
:1009C000E01CE42C640AE700E40803195E2D2E30D5
:1009D000E900E6206708E300E30364086302031C00
:1009E000F32C6408E300E3080319FB2C3030E90022
:1009F000E620E30BF62C6708E800640AE802031817
:100A0000802DD703640AE2006708E2026208E00072
:100A10006608DF0057080319122DE1000310DF0CF0
:100A2000E10B0E2D620803195E2D30305F07E900DF
:100A3000E6206008031D222DE40803195E2D2E30E8
:100A4000E900E620E003E20303195E2D57080319CD
:100A50002E2DE1000310DF0DE10B2A2D5F08E602C9
:100A60006608DB005808DC005908DD005A08DE0083
:100A70000310DA0DD90DD80DE60D0310DA0DD90DDE
:100A8000D80DE60D5E08DA07031C4B2DD90F4B2D50
:100A9000D80F4B2DE60A5D08D907031C522DD80F3D
:100AA000522DE60A5C08D8070318E60A5B08E60739
:100AB0000310DA0DD90DD80DE60D082D0000802D9C
:100AC0005E08DA07031C692DD90F692DD80F692D2F
:100AD000E60A5D08D907031C702DD80F702DE60AB1
:100AE0005C08D8070318E60A5B08E60700346608C6
:100AF000DB005808DC005908DD005A08DE0000342D
:100B0000000000345408D8005308D700D601550817
:100B100056020318B02D57080139D900580800397A
:100B2000DA00D908031D972DDA0803199D2DB83076
:100B30008316870083128714A22DB830831687008E
:100B4000831287100310D80CD70CB8308316870097
:100B5000831207158316870083120711D60A872D83
:100B600000340230D300A8204C08D8004B08D7002E
:100B70000621D601D501D4018F30D3007A08DA00DE
:100B80007908D9007808D8007708D7002421770899
:100B9000D3007808D4007908D5007A08D6004E082A
:100BA000D8004D08D700062183105608DE005508EE
:100BB000DD005408DC005308DB007A08E200790805
:100BC000E1007808E0007708DF009B217708D70074
:100BD0007808D8007908D9007A08DA0083107A08F2
:100BE000DE007908DD007808DC007708DB00E20130
:100BF000E101E0017F30DF009B217A08D200790813
:100C0000D1007808D0007708CF005208D6005108EC
:100C1000D5005008D4004F08D300DA01D9017A304A
:100C2000D8008830D7001C237708D3007808D40078
:100C30007908D5007A08D6002030E900E620560869
:100C4000DA005508D9005408D8005308D700DE014F
:100C5000DD010130DC008330DB0008240730D700E1
:100C600057085720D70AF700E900E6200B30570253
:100C7000031D302E0630D8002030E900E620D80BC6
:100C80003C2ED4016730D3000730D50082254E08B2
:100C9000D4004D08D3001030D50082254C08D40074
:100CA0004B08D3000A30D5008225B8308316870060
:100CB0008312071083168700831207140034B408C8
:100CC000031DF42F0130B4003108D8003008D700DC
:100CD0000621D601D501D4018F30D3007A08DA007D
:100CE0007908D9007808D8007708D7002421770838
:100CF000CB007808CC007908CD007A08CE00330804
:100D0000D8003208D700062183104E08DE004D08B7
:100D1000DD004C08DC004B08DB007A08E2007908B3
:100D2000E1007808E0007708DF009B217A08B9002D
:100D30007908B8007808B7007708B6003908CE00FF
:100D40003808CD003708CC003608CB00D201D101DD
:100D50004830D0008530CF00DD22031CB52EBD0108
:100D6000BC01BB017F30BA00332F3908CE003808F0
:100D7000CD003708CC003608CB00D201D1017A3043
:100D8000D0008830CF00DD22031CCD2EBD01BC0178
:100D90002030BB008230BA00332F3908CE0038082B
:100DA000CD003708CC003608CB00D2014030D1004E
:100DB0001C30D0008C30CF00DD22031CE62EBD019C
:100DC000BC014830BB008530BA00332F3908CE0053
:100DD0003808CD003708CC003608CB00D20150309F
:100DE000D1004330D0008F30CF00DD22031CFF2E16
:100DF000BD01BC017A30BB008830BA00332F3908FE
:100E0000CE003808CD003708CC003608CB00D20120
:100E10002430D1007430D0009230CF00DD22031C8A
:100E2000192FBD014030BC001C30BB008C30BA0013
:100E3000332F3908CE003808CD003708CC003608EB
:100E4000CB008030D2009630D1001830D0009730DF
:100E5000CF00DD22031C332FBD015030BC004330D6
:100E6000BB008F30BA00B830831687008312071E8C
:100E70006D2F83103908DE003808DD003708DC00EC
:100E80003608DB003D08E2003C08E1003B08E000DA
:100E90003A08DF009B217A08B9007908B800780881
:100EA000B7007708B600CE012430CD007430CC00F6
:100EB0009630CB003908D2003808D1003708D0006E
:100EC0003608CF00DD22031C6C2FB9012430B80096
:100ED0007430B7009630B6009E2F83143908DE00B8
:100EE0003808DD003708DC003608DB003D08E2008A
:100EF0003C08E1003B08E0003A08DF009B217A084B
:100F0000B9007908B8007808B7007708B600390842
:100F1000CE003808CD003708CC003608CB00D2010F
:100F2000D1012030D0008230CF00DD22031C9E2F63
:100F3000B901B8012030B7008230B6003908D600B8
:100F40003808D5003708D4003608D300DA01D901B3
:100F5000D8018F30D7001C237A08CE007908CD0045
:100F60007808CC007708CB00E8237908B10078082E
:100F7000B0003108D8003008D7000621D601D501CD
:100F8000D4018F30D3007A08DA007908D9007808C4
:100F9000D8007708D700242183143908DE003808E8
:100FA000DD003708DC003608DB007A08E20079084B
:100FB000E1007808E0007708DF009B217A08CE0086
:100FC0007908CD007808CC007708CB00E8237908B1
:100FD000B3007808B2003108CC003008CB003308E9
:0E0FE000CE003208CD00B1258A150A12DC2E93
:101000004B0DF700F70DF70DF830F7051F08C7393E
:1010100077049F002930F700F70B0C2800001F15FC
:101020001F19102883161E088312CC001E08CD003D
:101030004C08F8004D08F90000344F08D80050085B
:10104000D900DA01CC1F26285817D903CC174B0832
:101050000319C9287F304B02031C8528CB00DB0114
:101060000430DC000310CE0DCD0DCC0DDA0DDC0B01
:10107000322804304B020318452803304B02031D6D
:10108000BF280A305A02031CBF280330CB02DB0AF8
:1010900093210310CE0DCD0DCC0DDA0D7C21023045
:1010A000DC000310DA0CCC0CCD0CCE0CDC0B512880
:1010B00093210430DC000310CF0CD00CD10CD20CE7
:1010C000DC0B5B287C2193215108D2005008D10011
:1010D0004F08D000CF017C2193215008D2004F0847
:1010E000D100CF01D0017C21DA193928CB08031DAA
:1010F0007E28CE0ACD0ACC0ADA0ABF280310CE0D0C
:10110000CD0DCC0DDA0DCB033928CB09CB0A7F30BE
:10111000CB07DB010430DC000310CE0DCD0DCC0D70
:10112000DA0DDC0B8C280430CB0705304B02031C96
:10113000CB2893210310CE0DCD0DCC0DDA0D03106D
:10114000CE0DCD0DCC0DDA0D7C210310CE0DCD0DC5
:10115000CC0DDA0DDB0A0330DC000310DA0CCC0C0A
:10116000CD0CCE0CDC0BAD280330CB025A1E9528DB
:101170000310DA0CCC0CCD0CCE0CCB039528CB098C
:10118000CB0A0330CB075B0AD902031CD90101301B
:10119000CC280230CC280030D400D81BDA28D91B48
:1011A000DA28D9080319DA2820300C1ED52899002E
:1011B000D90BD428581FE0282D300C1EDD289900AB
:1011C000D81FED28D91BED28D9080319ED28303098
:1011D0000C1EE8289900D90BE428D8135813541C86
:1011E000F8285B08D4005B08D600580AD6072229E5
:1011F000D41CFC28580ADB00D80803197A292E30A1
:101200000C1E002999005B08D700D7035808570225
:10121000031C0C295808D700D708031915293030AA
:101220000C1E10299900D70B0F295B08DC00580A07
:10123000DC0203189C29CB03580AD6005B08D602AF
:101240005608D4005A08D3004B0803192C29D5009E
:101250000310D30CD50B2829560803197A293030EE
:1012600053070C1E312999005408031D3E29D80844
:1012700003197A292E300C1E3B299900D403D6037A
:1012800003197A294B0803194A29D5000310D30DF5
:10129000D50B46295308DA025A08CF004C08D00073
:1012A0004D08D1004E08D2000310CE0DCD0DCC0D4F
:1012B000DA0D0310CE0DCD0DCC0DDA0D5208CE0790
:1012C000031C6729CD0F6729CC0F6729DA0A51085B
:1012D000CD07031C6E29CC0F6E29DA0A5008CC0703
:1012E0000318DA0A4F08DA070310CE0DCD0DCC0D26
:1012F000DA0D222900009C295208CE07031C8529FB
:10130000CD0F8529CC0F8529DA0A5108CD07031C9A
:101310008C29CC0F8C29DA0A5008CC070318DA0A7A
:101320004F08DA0700345A08CF004C08D0004D08A7
:10133000D1004E08D2000034000000340130B5075F
:10134000CB0100207908C7007808C6004708D800FC
:101350004608D7008A1106218A154108CE004008A8
:10136000CD003F08CC003E08CB007A08D2007908B7
:10137000D1007808D0007708CF008A11DD228A15C5
:10138000031CD1294708D8004608D7008A11062136
:101390008A157A08C1007908C0007808BF0077086C
:1013A000BE000130CB0000207908C9007808C800D1
:1013B0004908D8004808D7008A1106218A1545082F
:1013C000CE004408CD004308CC004208CB007A0888
:1013D000D2007908D1007808D0007708CF008A11B0
:1013E000DD228A15031C032A4908D8004808D700C3
:1013F0008A1106218A157A08C5007908C400780880
:10140000C3007708C2003508783C03181C2BD601AE
:10141000D5014830D4008530D3004108DA004008B7
:10142000D9003F08D8003E08D7008A1124218A1528
:101430007708CB007808CC007908CD007A08CE0078
:10144000D6007908D5007808D4007708D300DA01EF
:10145000D901D8018930D7008A111C238A15770851
:10146000CF007808D0007908D1007A08D200831420
:101470007A08DE007908DD007808DC007708DB00F8
:10148000E201E1013030E0008530DF008A119B216C
:101490008A157A08C1007908C0007808BF0077086B
:1014A000BE00D601D5014830D4008530D3004508B0
:1014B000DA004408D9004308D8004208D7008A114E
:1014C00024218A157708CB007808CC007908CD0054
:1014D0007A08CE00D6007908D5007808D4007708BD
:1014E000D300DA01D901D8018930D7008A111C2331
:1014F0008A157708CF007808D0007908D1007A08DB
:10150000D20083147A08DE007908DD007808DC0058
:101510007708DB00E201E1013030E0008530DF00D8
:101520008A119B218A157A08C5007908C4007808B9
:10153000C3007708C2004108CE004008CD003F0834
:10154000CC003E08CB00D201D1010130D0000430E4
:10155000CF001D202C300C1EAB2A99004508CE0070
:101560004408CD004308CC004208CB00D201D10191
:101570000130D0000430CF001D200D300C1EBE2ADB
:1015800099000A300C1EC22A9900C030D3008A117B
:10159000A8208A152030E9008A11E6208A15410822
:1015A000DA004008D9003F08D8003E08D700DE0125
:1015B000DD010130DC008130DB008A1108248A154E
:1015C0002030E9008A11E6208A152030E9008A11CE
:1015D000E6208A154508DA004408D9004308D800F7
:1015E0004208D700DE01DD010130DC008130DB0084
:1015F0008A1108248A152030E9008A11E6208A150C
:101600006430E9008A11E6208A154230E9008A1127
:10161000E6208A150630CB002030E9008A11E6204A
:101620008A15CB0B0C2BB501C101C001BF01BE0156
:10163000C501C401C301C2018A150A12DE2EF701D9
:10164000F801510803105218F707F70CF80CD218DC
:10165000F707F70CF80C5219F707F70CF80CD2192A
:10166000F707F70CF80C521AF707F70CF80CD21A18
:10167000F707F70CF80C521BF707F70CF80CD21B06
:10168000F707F70CF80C8A150A129F2BCF01CD0132
:101690000A30CE00CC01CB080319542B4F08CF0AD7
:1016A0004B0784000008D00050082D3C031D612B1F
:1016B0000130CD004F08CF0A4B0784000008D0004E
:1016C0006B2B50082B3C031D6B2B4F08CF0A4B078D
:1016D00084000008D00050082F3C0318FA2B500853
:1016E000393C031CFA2B5008303C031D8E2B4B0851
:1016F0004F0784000008783C0319852B4B084F07DF
:1017000084000008583C031D8E2B1030CE00CF0AF9
:101710004F08CF0A4B0784000008D0004E080A3C4F
:10172000031DAB2B50082F3C0318AA2B5008393C43
:10173000031CAA2B0A30D1004C08D2001F2B3030DA
:1017400050027807CC004F08CF0A4B0784000008EE
:10175000D000922BFA2B4E08103C031DFA2B500898
:10176000603C0318BA2B50087A3C031CBA2B500873
:10177000DF39BB2B5008D00050082F3C0318C42B76
:101780005008393C0318CC2B5008403C0318FA2B66
:101790005008463C031CFA2B50082F3C0318DD2B45
:1017A0005008393C031CDD2B4C0ED100F030D10524
:1017B000303050025107CC00E62B4C0ED100F030F7
:1017C000D105413050020A3E5107CC004F08CF0AE4
:1017D0004B0784000008D0005008603C0318F72B2A
:1017E00050087A3C031CF72B5008DF39F82B5008BF
:1017F000D000BC2B4D0B022C4E080A3C031D022CC2
:10180000CC09CC0A4C08F8008A150A12F12E1030C7
:10181000F700FA01D601D30CD20C031C152C540886
:10182000FA070318D60A5508D607D60CFA0CF90C95
:10183000F80CF70B0B2C8A150A127B2CD001CE0169
:101840000A30CF00CD01CC01CB0803192D2C500854
:10185000D00A4B0784000008D10051082D3C031D1D
:101860003A2C0130CE005008D00A4B078400000803
:10187000D100442C51082B3C031D442C5008D00AA5
:101880004B0784000008D10051082F3C0318F12CAD
:101890005108393C031CF12C5108303C031D672CC6
:1018A0004B08500784000008783C03195E2C4B0855
:1018B000500784000008583C031D672C1030CF00EF
:1018C000D00A5008D00A4B0784000008D1004F0806
:1018D0000A3C031D8B2C51082F3C03188A2C5108FD
:1018E000393C031C8A2CD3010A30D2004D08D500A4
:1018F0004C08D400072C303051027807CC0079080E
:10190000CD000318CD0A5008D00A4B078400000808
:10191000D1006B2CF12C4F08103C031DF12C510809
:10192000603C03189A2C51087A3C031C9A2C5108ED
:10193000DF399B2C5108D10051082F3C0318A42CEF
:101940005108393C0318AC2C5108403C0318F12CC9
:101950005108463C031CF12C51082F3C0318C92C9C
:101960005108393C031CC92C4C0DD2004D0DD3003D
:10197000D20DD30DD20DD30DD20DD30DF030D20533
:10198000303051025207CC005308CD000318CD0A65
:10199000DE2C4C0DD2004D0DD300D20DD30DD20D47
:1019A000D30DD20DD30DF030D205413051020A3E95
:1019B0005207CC005308CD000318CD0A5008D00AB6
:1019C0004B0784000008D100603C0318EE2C51083E
:1019D0007A3C031CEE2C5108DF39EF2C5108D10062
:1019E0009C2C4F080A3C031DFC2C4E0BFC2CCC09F4
:1019F000CD09CC0A0319CD0A4C08F8004D08F900AE
:101A00000034CB0100207908C7007808C6004708D9
:101A1000D8004608D7008A1106218A157A08C10025
:101A20007908C0007808BF007708BE000130CB00FD
:101A300000207908C9007808C8004908D80048087B
:101A4000D7008A1106218A157A08C5007908C400D2
:101A50007808C3007708C200D601D5014830D40009
:101A60008530D3004108DA004008D9003F08D8008B
:101A70003E08D7008A1124218A157708CB00780800
:101A8000CC007908CD007A08CE00D6007908D500C0
:101A90007808D4007708D300DA01D901D801893059
:101AA000D7008A111C238A157708CF007808D00048
:101AB0007908D1007A08D20083147A08DE00790808
:101AC000DD007808DC007708DB00E201E10130305E
:101AD000E0008530DF008A119B218A157A08C10059
:101AE0007908C0007808BF007708BE00D601D5018C
:101AF0004830D4008530D3004508DA004408D900C6
:101B00004308D8004208D7008A1124218A15770893
:101B1000CB007808CC007908CD007A08CE00D6003A
:101B20007908D5007808D4007708D300DA01D90104
:101B3000D8018930D7008A111C238A157708CF0075
:101B40007808D0007908D1007A08D20083147A0886
:101B5000DE007908DD007808DC007708DB00E201B0
:101B6000E1013030E0008530DF008A119B218A15C9
:101B70007A08C5007908C4007808C3007708C20055
:101B80004108CE004008CD003F08CC003E08CB0005
:101B9000D201D1010130D0000430CF001D202C3003
:101BA0000C1ED02D99004508CE004408CD004308F6
:101BB000CC004208CB00D201D1010130D00004306A
:101BC000CF001D200D300C1EE32D99000A300C1E95
:101BD000E72D9900C030D3008A11A8208A15203043
:101BE000E9008A11E6208A154108DA004008D90088
:101BF0003F08D8003E08D700DE01DD010130DC00DF
:101C00008130DB008A1108248A152030E9008A110E
:101C1000E6208A152030E9008A11E6208A15450859
:101C2000DA004408D9004308D8004208D700DE0192
:101C3000DD010130DC008130DB008A1108248A15C7
:101C40002030E9008A11E6208A156430E9008A1103
:101C5000E6208A154230E9008A11E6208A1506300E
:101C6000CB002030E9008A11E6208A15CB0B312EFB
:101C70008A150A12462F84011F3083050630831609
:101C80009F004030990026309800903083129800D1
:101C9000A0010130A100A201A301A401A501A60198
:101CA000A701A801A901AA01AB01AC01AD01AE01D8
:101CB000AF01B001B101B201B301B401B501B0305F
:101CC00083168700B830870083120714003083160C
:101CD0008600FF30850083121F08383981389F0045
:101CE000813083169F008A118312C4288A15CB0184
:101CF0004B088A1104208A15CB0AF700E9008A11E3
:101D0000E6208A1510304B02031D782EC030D30018
:101D10008A11A8208A15B830831687008312871D80
:101D2000A12ECB014B088A1119208A15CB0AF70086
:101D3000E9008A11E6208A150B304B02031D922E12
:101D4000B02ECB014B088A1129208A15CB0AF70047
:101D5000E9008A11E6208A150B304B02031DA22EE2
:101D60000430CB00FA30CC008A1167208A15CB0BE7
:101D7000B22E8A1100298A15B4010330B3002A302B
:101D8000B200B101B001B830831687008312871DFD
:101D9000E12EB830831687008312871EDF2E0230B3
:101DA000CC008A1167208A15B83083168700831209
:101DB000871EDE2E8A115F2E8A159E29E02EB40121
:101DC000572F263084008403840A8C1EE52E1A08BF
:101DD00080000D300002031DE42E80012630CB0070
:101DE000462B7808CA004A08F700F7080319012FA4
:101DF000013077020319112F023077020319452FA2
:101E0000472FCB014B088A1139208A15CB0AF700DE
:101E1000E9008A11E6208A150A304B02031D022FC1
:101E2000572F263084008403840A8C1E152F1A082D
:101E300080000D300002031D142F80012630CB00DE
:101E40001E247908B1007808B0002630840084038D
:101E5000840A8C1E292F1A0880000D300002031DF1
:101E6000282F80012630CB001E247908B300780883
:101E7000B2003108CC003008CB003308CE00320865
:101E8000CD008A11B1258A15572F012D572FCB016F
:101E90004B088A1148208A15CB0AF700E9008A11FD
:101EA000E6208A150A304B02031D482F572FC32EF8
:021EB0006300CD
:02400E00723FFF
:00000001FF
